:1000000012C0AAC320C01FC01EC01DC01CC01BC080
:100010001AC07FC318C017C016C015C014C013C0C3
:1000200012C011C010C011241FBECFE5D4E0DEBF46
:10003000CDBF10E0A0E6B0E001C01D92AC38B10722
:10004000E1F7B5D293C3DCCF882309F4A2C0B89AF4
:1000500080916100882311F0C09A01C0C0988091FE
:10006000730090917400815F924014F08F9A07C0E2
:100070008F9A80916200882311F0979A01C0979817
:1000800080917300909174008B5D924014F08E9A71
:1000900007C08E9A80916300882311F0969A01C060
:1000A00096988091730090917400875C924014F050
:1000B0008D9A07C08D9A80916400882311F0959ADB
:1000C00001C095988091730090917400845B924078
:1000D00014F0BF9A07C0BF9A80916500882311F081
:1000E000C79A01C0C7988091730090917400825A9A
:1000F000924014F0BE9A07C0BE9A80916600882391
:1001000011F0C69A01C0C698809173009091740056
:100110008059924014F08C9A07C08C9A80916700A5
:10012000882311F0949A01C0949880917300909163
:1001300074008058924014F08B9A07C08B9A80917B
:100140006800882311F0939A01C0939880917300FE
:10015000909174008057924014F0899A07C0899A50
:1001600080916900882311F0919A01C09198809143
:100170007300909174008156924014F0889A07C0E1
:10018000889A80916A00882311F0909A0895909837
:100190000895B89AC098B89886B38F9A97988F9810
:1001A00080B38E9A96988E9880B38D9A95988D98F4
:1001B00080B3BF9AC798BF9886B3BE9AC698BE98B8
:1001C00086B38C9A94988C9880B38B9A93988B98DA
:1001D00080B3899A9198899880B3889A90988898E2
:1001E00080B30895882309F4A2C0B89A8091610071
:1001F000882311F0C09A01C0C0988091730090913B
:1002000074008A53934014F08F9A07C08F9A80919C
:100210006200882311F0979A01C09798809173002B
:10022000909174008052934014F08E9A07C08E9A79
:1002300080916300882311F0969A01C0969880916E
:100240007300909174008850934014F08D9A07C009
:100250008D9A80916400882311F0959A01C0959839
:100260008091730090917400815F924014F0BF9A66
:1002700007C0BF9A80916500882311F0C79A01C01A
:10028000C7988091730090917400875C924014F03D
:10029000BE9A07C0BE9A80916600882311F0C69A64
:1002A00001C0C6988091730090917400825A924068
:1002B00014F08C9A07C08C9A80916700882311F003
:1002C000949A01C094988091730090917400805822
:1002D000924014F08B9A07C08B9A80916800882313
:1002E00011F0939A01C093988091730090917400DB
:1002F0008156924014F0899A07C0899A80916900CA
:10030000882311F0919A01C0919880917300909187
:1003100074008654924014F0889A07C0889A80919D
:100320006A00882311F0909A089590980895B89AD9
:10033000C098B89886B38F9A97988F9880B38E9A02
:1003400096988E9880B38D9A95988D9880B3BF9A21
:10035000C798BF9886B3BE9AC698BE9886B38C9A43
:1003600094988C9880B38B9A93988B9880B3899A41
:100370009198899880B3889A9098889880B30895C6
:10038000DF93CF930F92CDB7DEB78A9882991AC0C8
:1003900010926D0010926C008091890090918A00FB
:1003A000895E914014F082E00AC0809189009091AA
:1003B0008A00019690938A008093890081E080935F
:1003C000720006C01092720010928A00109289008A
:1003D00080916C0090916D00895E91405CF080E0AE
:1003E00033DEA19AA99884EF91E090936D008093F9
:1003F0006C005DC080916C0090916D0001969093AF
:100400006D0080936C00A19AA99A94B3A09883E898
:1004100086B980E687B9198203C089818F5F898395
:1004200089818832D0F3369A3699FECF94BB24B1B5
:10043000229526952695237030E085B190E0880FAF
:10044000991F880F991F822B932B90937400809390
:10045000730010926100109262001092630010927B
:10046000640010926500109266001092670010926E
:1004700068001092690010926A00E0916000F0E05C
:10048000EF59FF4F81E08083A5989D9B02C0AADEB3
:1004900002C081E0D9DD80916000893018F01092AF
:1004A000600005C0809160008F5F809360000F90B6
:1004B000CF91DF910895A19AA99885B7806A85BFE9
:1004C00088958AEF90E00197F1F708950895E199F2
:1004D000FECFE199FECF1FBA1EBAE09A8DB38F37D7
:1004E00009F064C0E199FECFE199FECF81E090E090
:1004F0009FBB8EBBE09A8DB38F3709F057C0E1994F
:10050000FECFE199FECF82E090E09FBB8EBBE09AE8
:100510008DB38F3709F04AC0E199FECFE199FECF44
:1005200086E090E09FBB8EBBE09A8DB38F3709F0D9
:100530003DC0E199FECFE199FECF87E090E09FBBFF
:100540008EBBE09A8DB38F3709F030C0E199FECFB2
:10055000E199FECF88E090E09FBB8EBBE09A8DB31F
:100560008F3721F5E199FECFE199FECF83E090E04E
:100570009FBB8EBBE09A8DB380936F00E199FECF55
:10058000E199FECF84E090E09FBB8EBBE09A8DB3F3
:1005900080936B00E199FECFE199FECF85E090E07A
:1005A0009FBB8EBBE09A8DB380936E00089514BEFE
:1005B00088E10FB6F89481BD11BC0FBEA19AA99A2B
:1005C00010928B001092720010928A001092890093
:1005D00010926D0010926C008CE480936F0089E99A
:1005E00080936B008FEF80936E0071DF8FEF90E050
:1005F00097BD86BD82E18EBD8FB58C7B8FBD8FB5DB
:1006000080688FBDB99A1BBC1ABC83B7887F83BF33
:1006100083B7826083BF789489B7816089BF85B7CB
:10062000826085BF85B78E7F85BF78948BB78064E5
:100630008BBF4AEF50E073E031E062E080917200DE
:10064000813059F0823009F04DC02FC020E0CA013E
:100650000197F1F72F5F2233D1F78091720081303B
:10066000A9F380917200823049F380918B0082302F
:1006700061F0833091F0813009F780916B0090E058
:100680009BBD8ABD60938B00D9CF80916E0090E0B6
:100690009BBD8ABD70938B00D1CF80916F0090E09D
:1006A0009BBD8ABD30938B00C9CF80918B0088237E
:1006B00029F01BBC1ABC10928B000FC080916F00F8
:1006C00090E09BBD8ABD30938B0007C020E0CA013B
:1006D0000197F1F72F5F2233D1F7809172008230BA
:1006E000A9F3ACCF80918B00882309F0A7CF80912C
:1006F0006C0090916D00845F914009F09FCFA19AAA
:10070000A99885B7806A85BF8895CA010197F1F7D6
:1007100095CF1F920F920FB60F9211242F933F93F4
:100720004F935F936F937F938F939F93AF93BF93F9
:10073000EF93FF9325DEFF91EF91BF91AF919F91D2
:100740008F917F916F915F914F913F912F910F907A
:100750000FBE0F901F9018951F920F920FB60F9219
:1007600011240F900FBE0F901F901895F894FFCF93
:00000001FF
